:1000000042C0D5C15BC05AC059C058C057C056C0C5
:1000100055C054C053C052C051C050C04FC04EC054
:100020004DC04CC04BC04AC049C048C047C046C084
:1000300045C044C0040309041C037700770077001F
:100040002E00660069007300630068006C002E00DB
:10005000640065000E035500530042006100730008
:10006000700012011001FF000008C016DC0502013B
:1000700001020001090212000101008019090400B7
:1000800000000000000011241FBECFEFD2E0DEBF51
:10009000CDBF11E0A0E0B1E0E8E9FEE002C00590CC
:1000A0000D92A230B107D9F711E0A2E0B1E001C092
:1000B0001D92A334B107E1F7B1D4EDC6A1CFE9E6B3
:1000C000F0E0808183608083E89A08950F931F9306
:1000D000CF93DF9360912701161604F5635080914A
:1000E0002401C7E3D1E0C81BD109809123018D32DF
:1000F00009F44BC08091020187FD4CC0CE01A1D410
:100100008F3F09F483C0882309F458C030E020E011
:100110003093020120930001109227018091010188
:1001200084FF27C0809100018F3F19F1682F89302B
:10013000E0F5861B809300018091020180FD33C0B1
:100140000BE48F5F8093020187FD68C0662309F48A
:1001500054C088E191E016D5682F162F693008F455
:1001600079C08FEF809300019EE100931701909377
:1001700001019AE083B1837009F0F7C09150D1F783
:100180001092280110922201F0C08AE580930101AB
:100190006830B9F030E820E030930201209300018C
:1001A00010922701BBCF03ECCCCF68E0861B809375
:1001B00000018091020180FFC3CFF5CF30E02FEF27
:1001C000EBCF8881807609F05AC020E231E01092AE
:1001D00020018981882309F059C0109221013093B0
:1001E00026012093250130E822E08F818823A1F6A3
:1001F0008E81821788F6282FCFCF60E088E191E0CA
:10020000D2D094E08FEF80930001AFCF80930001B4
:100210008EE18093010130E02FEFBECF20912501C8
:100220003091260186FF1EC0462F41504F3F69F096
:10023000F901942FA8E1B1E084918D93319691500A
:10024000D8F72F5F3F4F240F311D309326012093A5
:10025000250183CF88E191E0A6D0912F9C5F1830D3
:1002600089F683CF462F41504F3F79F3F901942F00
:10027000A8E1B1E081918D939150E0F7E2CFCE01FA
:10028000CFD4282F8F3FA9F030E8AFCF853059F079
:100290008630B9F08830F9F0893031F18A3051F187
:1002A00030E820E0A2CF8A818093280130E820E066
:1002B0009CCF888187FD02C030E06ECF2E8130E078
:1002C0006BCF8B818130E9F0823081F1833011F185
:1002D00030EC20E08ACF8AE291E09093260180936F
:1002E000250130E821E081CF8A8180932A0130E81E
:1002F00020E07BCF309326012093250130E821E0D8
:1003000074CF82E690E0909326018093250130EC33
:1003100022E16BCF8A81882391F484E390E090936B
:1003200026018093250130EC24E05FCF84E790E044
:10033000909326018093250130EC22E156CF813045
:1003400059F0823029F684E590E09093260180935D
:10035000250130EC2EE049CF88E390E09093260110
:100360008093250130EC2CE140CFDF91CF911F919C
:100370000F910895A82FB92F8FEF9FEF41E050EA1A
:10038000615070F02D9138E0722F782796958795FF
:10039000269570FF02C0842795273A95A9F7F0CFDC
:1003A000809590950895E6DF8D939D930895CF9362
:1003B000CFB7CF93189BFECF189B09C0189B07C0DF
:1003C000189B05C0189B03C0189B01C09EC0DF93FB
:1003D000C0912401DD27C55DDE4F189B02C0DF916F
:1003E000EBCF2F930F931F9303B12FEF00FB20F957
:1003F0004F933F9313B14FEF012700FB21F93BE0EF
:1004000031C04E7F012F13B1216028C0102F4D7FC6
:100410002260000003B129C04B7F2460012F00003F
:1004200013B12BC013B1477F28602AC04F7E03B1A0
:1004300020612CC04F7D13B120622FC04F7B03B1D0
:10044000206432C0422703B149934FEF00001027C8
:1004500010FB20F913B11370A9F1297F91F2012744
:1004600000FB21F903B1237F89F23150F0F110270D
:1004700010FB22F913B1277E79F2012700FB23F943
:100480002F7C81F203B1102710FB24F92F7971F230
:1004900000C013B1012700FB25F92F7359F200C0EA
:1004A00003B1102710FB26F9223040F200C013B12F
:1004B000012700FB27F9243028F64F77206813B175
:1004C0000000F9CF3B503195333011E01CBBB8F040
:1004D000C31BD0400881033C41F10B3431F1198139
:1004E000412F1F7720912201121731F4093691F123
:1004F0000D3279F0013E69F02227209329013F91C6
:100500004F911F910F912F91DF91CF91CFBFCF913D
:100510001895009329013F914F911F910F912F91B1
:10052000DF91CCB3C0FD46CFF0CF0091290100236D
:1005300031F310912701112349F534304AF13093FA
:10054000270100932301109124013BE0311B3093DC
:1005500024011EC0009127010130C4F40AE5309146
:10056000010134FD17C000930101C7E1D1E016C0BD
:10057000052710E005B91FC0052722C0052727C0A1
:1005800005272CC0052710E005B933C04AE503C094
:1005900042ED01C0432FC4E1D0E032E014B113605A
:1005A000289A05B114B95F9353E020E820FF05278E
:1005B00005B9279517951C3FD8F620FF05272795E5
:1005C00005B917951C3FC0F620FF052727951795FD
:1005D00005B91C3F98F620FF0527279517951C3F66
:1005E00005B970F600C0499120FF052705B9279588
:1005F00017951C3F38F620FF0527279505B9179555
:100600001C3F38F520FF05272795179505B91C3F96
:1006100010F520FF0527279517951C3F05B9E8F42D
:10062000242F3A9519F60C7F5F9105B900C01091FF
:100630002801C651D04011F01093220111E01CBBDB
:10064000016014B11C7F402F4C7F05B914B945B926
:1006500056CF0527D3CF0527D8CF0527DDCF3B9829
:10066000439A00000000339904C082E58CBD1DBC94
:1006700008953A9A429800000000339B07C082E533
:100680008CBD81E08DBD3A98429A089583E58CBD7A
:100690001DBC3A98429A0895882339F481E893E082
:1006A000909342018093410108958EE993E09093E5
:1006B000420180934101089596B586B5891B8C301F
:1006C000E0F308952C9A3D9A459884B18C6284B9E0
:1006D0002A982D98F1DF2A9AEFDF2A98809141011C
:1006E000909142018E59934009F00895B8DF089522
:1006F00084B1837D84B985B1837D85B93D981CBC67
:100700000895FF920F931F93182FFF2400E00CC051
:100710002B98FF0C1C99F394CFDF2D9ACDDF2D98E9
:100720000F5F083029F0110F17FFF2CF2B9AF1CF8E
:100730008F2D90E01F910F91FF9008958EBD0DB405
:1007400007FEFDCF8EB590E008950F931F930FE144
:1007500003C001500F3F51F1E0914101F09142017E
:100760008CEA0995E0914101F091420183E50995F8
:10077000E0914101F091420180E00995182FE0914C
:100780004101F091420180E00995133591F01CBCC4
:100790002D9A92DF2D9890DF809141019091420136
:1007A0008E599340B1F65BDF0150B0F681E090E0E6
:1007B00002C080E090E01F910F910895EF92FF92A8
:1007C0000F931F937B018C01862F8170880F880FF8
:1007D000880FE0914101F091420180620995D801B2
:1007E000C70129E0B695A795979587952A95D1F7E2
:1007F000E0914101F0914201099516950795F79412
:10080000E794E0914101F09142018E2D0995E0912C
:100810004101F091420180E0099590E01F910F9114
:10082000FF90EF9008950F931F938C01E091410189
:10083000F091420180EA0995812F9927E0914101C9
:10084000F09142010995E0914101F0914201802F20
:100850000995E0914101F091420180E0099590E015
:100860001F910F910895FF920F931F938C01F62E05
:10087000E0914101F091420180EC0995812F992787
:10088000E0914101F09142010995E0914101F0911F
:100890004201802F0995E0914101F09142018F2D95
:1008A00009958EE1AED080E090E01F910F91FF900E
:1008B0000895CF92DF92EF92FF920F931F936B01F7
:1008C0007C01142FE0914101F09142018CE40995E3
:1008D000E0914101F0914201D701C60169E0B6956E
:1008E000A795979587956A95D1F70995E09141016C
:1008F000F0914201D701C601B695A79597958795C6
:100900000995E0914101F091420180E009951F3F76
:10091000A9F006B51EE1C701B60150DF8F3F59F4BB
:1009200086B5801B8D3310F006B51150112399F751
:1009300081E090E007C080E090E004C08FE061D0EB
:1009400080E090E01F910F91FF90EF90DF90CF90AB
:100950000895CF92DF92EF92FF920F931F936B0156
:100960007C01042F122FE0914101F0914201862F6A
:100970008170880F880F880F80640995E09141018C
:10098000F0914201D701C60129E0B695A795979548
:1009900087952A95D1F70995E0914101F09142019F
:1009A000D701C601B695A795979587950995E091CA
:1009B0004101F0914201802F09951123A1F00F37D9
:1009C000A9F006B51EE1C701B601F8DE8F3759F46C
:1009D00086B5801B8D3310F006B51150112399F7A1
:1009E00081E090E007C080E090E004C08FE009D093
:1009F00080E090E01F910F91FF90EF90DF90CF90FB
:100A00000895382F882349F020E096B586B5891BD4
:100A10008C33E0F32F5F2317C1F708951BB815B887
:100A20008BEF8AB98FEF84B914B893E097B98EEF42
:100A300088B995BD81E030DE42DB789447DB46DB48
:100A4000FDCFFF920F931F93CF93DF93062F20913B
:100A50000301213029F0243019F08FEF90E08CC091
:100A6000002309F487C0EC01FF2410E051C08091FD
:100A7000130190911401892B09F057C060910F0167
:100A8000709110018091110190911201488161DFF4
:100A90008091040190910501019790930501809345
:100AA0000401892BE1F4109203018091150181FF6B
:100AB00039C08091160190E020911301309114010A
:100AC0008217930779F160910F0170911001809165
:100AD0001101909112014881ECDEFF24F394809182
:100AE0000F0190911001A0911101B0911201019696
:100AF000A11DB11D80930F0190931001A0931101CE
:100B0000B09312011F5F2196101789F12091030104
:100B1000213009F4ACCF688180910F0190911001D0
:100B2000A2DEB6CFFF24F394DACF60910F0170916B
:100B30001001809111019091120120E0488109DF9C
:100B400080911601815080931601882309F0A0CF6F
:100B500060910F017091100180911101909112012B
:100B60004881A7DE809113018093160191CF8F2DCC
:100B700090E002C080E090E0DF91CF911F910F9153
:100B8000FF9008950F931F93CF93DF93AC01062F2F
:100B900020910301822F8250823018F08FEF90E075
:100BA0003AC06623A1F1EA0110E01FC080910F0155
:100BB0009091100138DE888380910F01909110018F
:100BC000A0911101B09112010196A11DB11D809358
:100BD0000F0190931001A0931101B09312011F5FB8
:100BE0002196101779F0209103012230F9F66091D7
:100BF0000F01709110018091110190911201DEDDC1
:100C00008883DACF083018F0802F90E004C010926B
:100C10000301802F90E0DF91CF911F910F910895F4
:100C2000CF93DF93EC018981813041F1823009F467
:100C3000CBC0833009F4CDC0843059F1873009F43A
:100C400099C0853009F418C1863009F44FC0883046
:100C500009F4E2C0893079F481E0809306018A8149
:100C60009B81AC81BD8180930F0190931001A09373
:100C70001101B093120120E030E003C1329933C07A
:100C800080E00ADD1092060141981CDD20E030E092
:100C9000F8C0809106018823A1F48B8190E0982F01
:100CA00088272A8130E0822B932BAA2797FDA095D5
:100CB000BA2F80930F0190931001A0931101B0936C
:100CC00012018F8190E0982F88272E8130E0822BAF
:100CD000932B909305018093040182E0809303019C
:100CE0002FEF30E0CEC081E0D7DCCCCF8091060181
:100CF0008823A1F48B8190E0982F88272A8130E007
:100D0000822B932BAA2797FDA095BA2F80930F01D2
:100D100090931001A0931101B09312018C819D81D9
:100D2000292F2F7020931501492F50E0407F5070DC
:100D300042955295507F5427407F5427480F511DAC
:100D4000509314014093130120FF02C040931601F9
:100D50008F8190E0982F88272E8130E0822B932B73
:100D6000909305018093040181E0809303012FEFAC
:100D700030E087C0809106018823A1F48B8190E048
:100D8000982F88272A8130E0822B932BAA2797FD62
:100D9000A095BA2F80930F0190931001A093110199
:100DA000B09312018F8190E0982F88272E8130E038
:100DB000822B932B909305018093040183E0809311
:100DC00003012FEF30E05DC093DC419A20E030E07A
:100DD00058C0E0914101F09142018A8109958093C8
:100DE0000701E0914101F09142018B8109958093C7
:100DF0000801E0914101F09142018C8109958093B5
:100E00000901E0914101F09142018D8109958093A2
:100E10000A0124E030E035C0809106018823A1F466
:100E20008B8190E0982F88272A8130E0822B932BAA
:100E3000AA2797FDA095BA2F80930F0190931001D8
:100E4000A0931101B093120110921401109213019A
:100E5000109215018F8190E0982F88272E8130E025
:100E6000822B932B909305018093040184E080935F
:100E700003012FEF30E005C068DC8093070121E01B
:100E800030E087E091E09093260180932501C9012D
:080E9000DF91CF910895FFCF1F
:020E9800FF5AFF
:00000001FF
